:020000020000FC
:100000000C9404000C942B000FE50DBF04E00EBF10
:100010000E94AE000E94BE000E9451000E94E900B2
:100020000E9494000FEF0E9401010E941F0029F41A
:1000300004E60E94F0000E94BE000C940C000091A7
:10004000600010916200011729F400916100109185
:100050006300011708950F930FB70F931F93FF933A
:10006000EF9300916A00039500936A0000E008BBDB
:1000700000916400029502BB0295F0E0E5E6E00F16
:100080000024F01D108118BB0395053009F40027EA
:1000900000936400EF91FF911F910F910FBF0F919B
:1000A000189520E027B910E816B9369A3699FECF90
:1000B00015B1213089F0133041F0103059F400911E
:1000C00060000A950093600005C0009160000395F0
:1000D0000093600021E0E6CF133041F0103059F476
:1000E000009161000A950093610005C000916100D4
:1000F0000395009361000E947E00089500916000C6
:1001000017E00E948D00009360000091610015E0EF
:100110000E948D0000936100089500601AF001179D
:1001200011F4025003950895FF27E0E60E949D0018
:10013000FF27E2E60E949D00089511910E94A7000A
:100140001081E5E6E10F1081102B1083089501E086
:100150001A951AF0000F0C94A80008950AE005BF44
:1001600000EC0BBF00E007B900E806B900E80ABBE5
:100170000FEF07BB00EF01BB7894089500E00093F8
:10018000600002E0009361000F920F920E94D10084
:100190000F91009362000F91009363000E94E900A9
:1001A00008950EB7F02F0DB7E02F00916A00102FC1
:1001B0001770153008F0155014830295102F177022
:1001C000123010F413951395173008F0155013835F
:1001D000089505E0F0E0E5E601920A95E9F7089553
:1001E00010E81BBB0F9305E00E9401010F9110E086
:1001F0001BBB0F9305E00E9401010F910A9581F747
:100200000895C79A1FEF1A95F1F70A95D9F7C7987D
:0202100008954F
:00000001FF
